:1000000012C02AC029C028C027C026C025C08EC063
:1000100023C022C021C020C01FC01EC01DC01CC0E4
:100020001BC01AC019C011241FBECFEDCDBF10E0F8
:10003000A0E6B0E0E2ECF2E002C005900D92A23939
:10004000B107D9F710E0A2E9B0E001C01D92A739CD
:10005000B107E1F716D133C1D3CF5D9BFECF8CB989
:100060000895FC019DE009C05D9BFECF8CB98A30EC
:1000700019F45D9BFECF9CB9319680818823A1F74E
:100080000895E82FF0E0EC56FF4F6083813039F09F
:10009000813018F0823061F407C066BF0895862F62
:1000A00090E099BD88BD0895862F90E09BBD8ABDE4
:1000B0000895E4E9F0E0E80FF11D80810895809350
:1000C000940086BF6093950070E079BD68BD409351
:1000D000960050E05BBD4ABD0895882321F4E0E618
:1000E000F0E09DE01CC017BA969AEEE6F0E09DE0C5
:1000F00009C05D9BFECF8CB98A3019F45D9BFECFA1
:100100009CB9319680818823A1F708955D9BFECF2D
:100110008CB98A3019F45D9BFECF9CB931968081F1
:100120008823A1F78EE187BB969808951F920F92BE
:100130000FB60F9211242F933F934F935F936F93BA
:100140007F938F939F93AF93BF93EF93FF938CB164
:1001500090919300913009F446C0913020F0923094
:1001600009F061C046C0873651F1883640F48133CA
:1001700081F0823669F1803309F055C008C08237BA
:10018000B9F08F3F71F18F3609F04DC005C080E0A6
:1001900001C081E0A2DF47C01092940016BE109209
:1001A000950019BC18BC109296001BBC1ABC3BC031
:1001B0008091940080958093940086BF34C0809194
:1001C000950080958093950090E099BD88BD2BC0E7
:1001D0008091960080958093960090E09BBD8ABDAB
:1001E00022C081E003C08093920082E0809393005C
:1001F0001AC090919200973649F0923719F09236D2
:1002000081F40AC08093940086BF0BC08093950050
:1002100090E099BD88BD05C08093960090E09BBD9D
:100220008ABD10929300FF91EF91BF91AF919F9182
:100230008F917F916F915F914F913F912F910F908F
:100240000FBE0F901F90189512BA18BA80E481BBA8
:1002500080E043DF12B88FE089B988E98AB981E884
:1002600080BF91E093BF1CBE8CB786BF81EA8FBD73
:100270009EBD19BC18BC88B599B59BBD8ABD789444
:100280000895E2DFEBE7F0E09DE009C05D9BFECF63
:100290008CB98A3019F45D9BFECF9CB93196808170
:1002A0008823A1F78EEF8093940086BF109295006B
:1002B00019BC18BC109296001BBC1ABCFFCFF89456
:0202C000FFCF6E
:1002C2005049432064697361626C65640A00504955
:1002D2004320656E61626C65640A0044696F6465FF
:1002E2007220436F6E74726F6C20302E302E310A82
:0202F20000000A
:00000001FF
